:1000000083160C3085000030860083126228820738
:100010003E344134413441343E34003410342034D1
:100020007F3400342734493449344934313422345C
:1000300041344934493436340C34143424347F3454
:1000400004347A3449344934493446343E344934EA
:1000500049344934263440344734483450346034C9
:1000600036344934493449343634323449344934E5
:1000700049343E3400348514000085101108860090
:100080004E20120886004E20130886004E201408C9
:1000900086004E20150886004E2008009B0B4E2837
:1000A0000030860005100000051408000530980097
:1000B00011308400170807208000840A970A980BE3
:1000C0005A2808000030970056209E123B20051D3C
:1000D0006A2865289E1A66281708323A031D722876
:0A00E0000030970056209E16662897
:00000001FF
